S12301000000000000000000000000000000000000000000000000000000000000000000DB
S1210120000000000000000000000000000000000000000000000000000000000000BD
S12350007E508A7E50C67E50D57E50E47E50F37E51007E51647E51CB7E51E87E51EE7E51AB
S1235020F47E51F57E52007E52197E521F7E52257E52347E523F7E526B7E52EF7E53017EBA
S1235040534C7E534D7E534E7E534F70726F6772616D2061382E61736D20342D32362D39E1
S1235060342020686331312064617461206C6F6720746F207063202033206279746573209F
S1235080393630302062617564048E00FF8680B710398630B7102BBD5234CE504BBD52EF98
S12350A0BD51F5BD51F5BD51CB010101BD50F38603BD5255B61031BD5255B61032BD525566
S12350C0BD522520E739CE003218CE164E180926FC0926F539CE00FA18CE164E180926FC19
S12350E00926F539CE01F418CE164E180926FC0926F539CE10308614A7001F0080FC4F3930
S123510018CE000ACC0000FD025ACC0000FD025CCC0000FD025ECC0000FD0260BD50F3F605
S123512010314FFD0258FC025AF30258FD025AF610324FFD0258FC025CF30258FD025CF6B0
S123514010334FFD0258FC025EF30258FD025EF610344FFD0258FC0260F30258FD0260185A
S12351600926B939C640F71023FC1018F30113FD1018FE012D09FF012D27013BFE012FFF98
S1235180012DC680F71039CE10308614A7001F0080FC4FFE0129B61031A700FC0129C3006F
S12351A001FD0129FE0129B61032A700FC0129C30001FD0129FC0129B301271A8300002E1F
S12351C0022006FC0125FD01293B39CE00D918CE51F4867EA7001AEF01CE00DC18CE51641A
S12351E0867EA7001AEF0139C680F7103939C600F71007393B860DBD5255860ABD52553992
S1235200CE1031BDFFBECE1032BDFFBECE1033BDFFBECE1034BDFFBE398630B7102B3986C0
S123522031B7102B39CE000118CE05DC180926FC0926F5398600B7102C862CB7102D39A6DA
S1235240008D04A600200444444444840F8B3081392F028B07F6102EC4C0C1C026F7F610B8
S123526000C404270220EEB7102F39CE528018CE00C4C63CA60018A7000818085A26F53975
S12352807E53017E52BC7E52BC7E52BC7E52BC7E52BC7E52BC7E52BC7E52BC7E52BC7E527C
S12352A0DC7E52D87E52BC7E52E07E52C07E52D47EE8E47E52C87E52CC7E52D0860120240D
S12352C0860220208603201C8604201886052014860620108607200C8608200886092004DE
S12352E0860A2000B7020AB6020ABD524B20F8BD51F536A60081042706BD52550820F432C0
S123530039F6102EB6102FC4082635F602252615812F2610B60220B7022184EFB70220863E
S123532003B702253B7A02252608810D26181420043BF602255A2604B702263BB702273B69
S12353408601B702243B8602B702243B393939393C3736CE03178630A100261B8D3F201DF4
S1235360A10026198D378D3509A100261B8D2EA100261B8D28201DA600BDFFB808A600BDC4
S1235380FFB8862EBDFFB808A600BDFFB808A600BDFFB808A600BDFFB8323338393608862A
S12353A020BDFFB832393C3736EC00CE2710028FCB30F703178FCE03E8028FCB30F70318CD
S12253C08FCE0064028FCB30F703198FCE000A02CB30F7031B8FCB30F7031A323338397D
S9030000FC
